:10000000B601FD280408A700861006100610831606
:100010008610061006100F30860583122708B618C2
:100020002F283A30A10098308E203330A60043208C
:100030001330A10088308E20432064308D2043206F
:1000400064308D202230A600432028302E200C3032
:100050002E2006302E20B61427082F283614A6008E
:10006000361C3D280610033C031C42284220073062
:10007000A100D0308E20031408003614FE3C031972
:10008000F8280614361C361086140F30860526080C
:10009000F03986048610A60E3618432832308D209B
:1000A00003140800B71329080319B7170530A8006F
:1000B0002730A300103068200330A300E830682008
:1000C000A30164306820A3010A30682024086F2847
:1000D000A2002508A1002408A000D1202008A0002B
:1000E000A8030319B713290803197928280203184C
:1000F00008002008031DB713B71B0800303EF32883
:10010000A301A200FF30A207031CA307031CF828C9
:100110000330A100DF308E208228A101E83EA0003C
:10012000A109FC30031C9728A00703189428A007F6
:100130006400A10F942820189D28A01CA12800006D
:10014000A1280800A000A11BED202008F82803101A
:10015000A10CA00CFF3E0318A7282008F828A10135
:10016000A301A2000230BA28A2000330BA28A200DC
:100170000630BA28A80023082102031DC12822083E
:100180002002043003180130031902302805031D32
:10019000FF30F8280038031DFF300405031DFF3031
:1001A000F8281030A600A501A401210DA40DA50D6D
:1001B0002208A4022308031C230FA5020318E72822
:1001C0002208A40723080318230FA5070310A00D76
:1001D000A10DA60BD5282008F828A009A109A00A7E
:1001E0000319A10A0800840031088A00300882003F
:1001F00083130313831264000800831607309F00E3
:10020000643083128020FE300320013003208316E7
:10021000051585158312FA30C000C1019230BC006B
:10022000FF30BD00FA30C200C3019230BE00FF3083
:10023000BF00FE3003200130032020300320203097
:1002400003202030032020300320203003204430BE
:1002500003204F30032055300320423003204C3020
:10026000032045300320203003202030032020309D
:1002700003202030032020300320FE300320C03034
:100280000320203003202030032054300320483046
:10029000032045300320523003204D3003204F30DF
:1002A00003204D30032045300320543003205230CA
:1002B000032045300320203003202030032020304D
:1002C00003200330A300E83081208A110A1290270E
:1002D0008A110A12CC30CA008A150A1211208A111A
:1002E0000A12CC30CA008A150A1236208A110A1264
:1002F0004430CA008A150A1211208A110A124430A9
:10030000CA008A150A1236208A110A120730A30081
:10031000D03081208A110A1290278A110A12CC301B
:10032000CA008A150A1211208A110A12CC30CA009A
:100330008A150A1236208A110A12BE30CA008A159E
:100340000A1211208A110A128A150A128D208A11A6
:100350000A12BE30CA008A150A1236208A110A1201
:100360008A150A12A4208A110A120030C91B013012
:10037000A0000030AF20B2000030BF1B0130A00051
:100380000030AF20B400320884003408CA20B40022
:10039000B5006400340835048A110A120319E429EF
:1003A0008A110A124808A0004908A1003F08A300CA
:1003B0003E08B7208A110A12031DE4298A110A1285
:1003C0004808BE004908BF000030C91B0130A0002A
:1003D0000130AF20B2000030BF1B0130A00001305F
:1003E000AF20B400320884003408CA20B400B5003D
:1003F0006400340835048A110A120319212A8A116B
:100400000A124908A1004808A220B2002108B3003E
:100410003F08A1003E08A220B4002108B500320820
:10042000A0003308A1003508A3003408B4208A11C5
:100430000A12031D212A8A110A124808BE0049081F
:10044000BF000030C91B0130A0000030AF20B20057
:100450000030BF1B0130A0000130AF20B4003208D3
:1004600084003408CA20B400B500640034083504A0
:100470008A110A120319422A8A110A124808BE0078
:100480004908BF000030C91B0130A0000030AF2078
:10049000B2000030C31B0130A0000030AF20B40018
:1004A000320884003408CA20B400B500640034085F
:1004B00035048A110A120319712A8A110A1248088E
:1004C000A0004908A1004308A3004208B4208A11F3
:1004D0000A12031D712A8A110A124808C20049082B
:1004E000C3000030C91B0130A0000130AF20B200B2
:1004F0000030C31B0130A0000130AF20B40032082F
:1005000084003408CA20B400B500640034083504FF
:100510008A110A120319AE2A8A110A124908A10087
:100520004808A220B2002108B3004308A1004208F5
:10053000A220B4002108B5003208A0003308A100B1
:100540003508A3003408B7208A110A12031DAE2A09
:100550008A110A124808C2004908C3000030C91BAA
:100560000130A0000130AF20B2000030C31B0130C9
:10057000A0000030AF20B400320884003408CA2044
:10058000B400B5006400340835048A110A12031956
:10059000CF2A8A110A124808C2004908C300640021
:1005A0008A110A12C91F1B2B8A110A124908A100BD
:1005B0004808A220C8002108C900FE3003200130ED
:1005C0000320203003205430032020300320493002
:1005D00003206E30032074300320203003202D30A0
:1005E0000320A9010310490CB300480CB2003208E3
:1005F000A4003308A5000230B000B10152202C3015
:100600000320A9010530481C0301B2000030481C3A
:100610000301B3003208A4003308A5000230B00083
:10062000B101522020300320DF300320433003206B
:100630008A110A12562BFE3003200130032020308D
:1006400003205430032020300320493003206E3033
:100650000320743003202030032020300320A90120
:100660000310490CB300480CB2003208A400330850
:10067000A5000230B000B10152202C300320A901A6
:100680000530481C0301B2000030481C0301B300D0
:100690003208A4003308A5000230B000B101522096
:1006A00020300320DF300320433003200030C71BFD
:1006B0000130A0000030AF20B2000030BD1B01307F
:1006C000A0000030AF20B400320884003408CA20F3
:1006D000B400B5006400340835048A110A12031905
:1006E000852B8A110A124608A0004708A1003D0880
:1006F000A3003C08B7208A110A12031D852B8A111A
:100700000A124608BC004708BD000030C71B013074
:10071000A0000130AF20B2000030BD1B0130A000AE
:100720000130AF20B400320884003408CA20B4007D
:10073000B5006400340835048A110A120319C22B6B
:100740008A110A124708A1004608A220B200210817
:10075000B3003D08A1003C08A220B4002108B50068
:100760003208A0003308A1003508A3003408B420E3
:100770008A110A12031DC22B8A110A124608BC00F4
:100780004708BD000030C71B0130A0000030AF207B
:10079000B2000030BD1B0130A0000130AF20B4001A
:1007A000320884003408CA20B400B500640034085C
:1007B00035048A110A120319E32B8A110A1246081A
:1007C000BC004708BD000030C71B0130A00000304E
:1007D000AF20B2000030C11B0130A0000030AF20BC
:1007E000B400320884003408CA20B400B5006400A4
:1007F000340835048A110A120319122C8A110A12BC
:100800004608A0004708A1004108A3004008B42002
:100810008A110A12031D122C8A110A124608C000FE
:100820004708C1000030C71B0130A0000130AF20D5
:10083000B2000030C11B0130A0000130AF20B40075
:10084000320884003408CA20B400B50064003408BB
:1008500035048A110A1203194F2C8A110A1247080B
:10086000A1004608A220B2002108B3004108A1005F
:100870004008A220B4002108B5003208A0003308C7
:10088000A1003508A3003408B7208A110A12031DFD
:100890004F2C8A110A124608C0004708C1000030D8
:1008A000C71B0130A0000130AF20B2000030C11BD7
:1008B0000130A0000030AF20B400320884003408BA
:1008C000CA20B400B5006400340835048A110A1245
:1008D0000319702C8A110A124608C0004708C1008B
:1008E00064008A110A12C71FBC2C8A110A12470819
:1008F000A1004608A220C6002108C700FE30032040
:10090000C030032020300320543003202030032047
:10091000453003207830032074300320203003203A
:100920002D300320A9010310470CB300460CB20080
:100930003208A4003308A5000230B000B1015220F3
:100940002C300320A9010530461C0301B200003001
:10095000461C0301B3003208A4003308A50002308E
:10096000B000B101522020300320DF30032043309B
:1009700003208A110A12F72CFE300320C030032016
:100980002030032054300320203003204530032042
:1009900078300320743003202030032020300320DF
:1009A000A9010310470CB300460CB2003208A400A2
:1009B0003308A5000230B000B10152202C300320D2
:1009C000A9010530461C0301B2000030461C03019A
:1009D000B3003208A4003308A5000230B000B10112
:1009E000522020300320DF30032043300320073023
:1009F000A300D030812064008A110A1205192E2F1D
:100A00008A110A1264008A110A12C31F4E2D8A111C
:100A10000A124308A1004208A220C4002108C50010
:100A2000FE300320023003204D30032069300320C4
:100A30006E30032020300320493003206E30032025
:100A4000203003202D300320A9010310450CB300F2
:100A5000440CB2003208A4003308A5000230B000F4
:100A6000B10152202C300320A9010530441C0301A0
:100A7000B2000030441C0301B3003208A400330864
:100A8000A5000230B000B101522020300320DF3039
:100A90000320433003208A110A12892DFE300320DF
:100AA000023003204D300320693003206E300320D4
:100AB00020300320493003206E30032020300320F3
:100AC00020300320A9010310430CB300420CB200F4
:100AD0003208A4003308A5000230B000B101522052
:100AE0002C300320A9010530421C0301B200003064
:100AF000421C0301B3003208A4003308A5000230F1
:100B0000B000B101522020300320DF3003204330F9
:100B100003200730A300D030812064008A110A121C
:100B2000BF1FD92D8A110A123F08A1003E08A2203A
:100B3000C4002108C500FE300320023003204D30E0
:100B40000320613003207830032020300320493017
:100B500003206E300320203003202D300320A90114
:100B60000310450CB300440CB2003208A400330853
:100B7000A5000230B000B10152202C300320A901A1
:100B80000530441C0301B2000030441C0301B300D3
:100B90003208A4003308A5000230B000B101522091
:100BA00020300320DF300320433003208A110A1253
:100BB000142EFE300320023003204D30032061301C
:100BC00003207830032020300320493003206E308A
:100BD00003202030032020300320A90103103F0C04
:100BE000B3003E0CB2003208A4003308A500023066
:100BF000B000B10152202C300320A90105303E1C69
:100C00000301B20000303E1C0301B3003208A4000F
:100C10003308A5000230B000B1015220203003207B
:100C2000DF300320433003200730A300D030812081
:100C300064008A110A12C11F642E8A110A12410827
:100C4000A1004008A220C4002108C500FE300320F6
:100C5000C03003204D300320693003206E30032064
:100C6000203003204530032078300320203003203B
:100C70002D300320A9010310450CB300440CB20031
:100C80003208A4003308A5000230B000B1015220A0
:100C90002C300320A9010530441C0301B2000030B0
:100CA000441C0301B3003208A4003308A50002303D
:100CB000B000B101522020300320DF300320433048
:100CC00003208A110A129F2EFE300320C030032019
:100CD0004D300320693003206E3003202030032084
:100CE00045300320783003202030032020300320BB
:100CF000A9010310410CB300400CB2003208A4005B
:100D00003308A5000230B000B10152202C3003207E
:100D1000A9010530401C0301B2000030401C030152
:100D2000B3003208A4003308A5000230B000B101BE
:100D3000522020300320DF300320433003200730CF
:100D4000A300D030812064008A110A12BD1FEF2E4B
:100D50008A110A123D08A1003C08A220C400210803
:100D6000C500FE300320C03003204D300320613029
:100D700003207830032020300320453003207830D2
:100D80000320203003202D300320A9010310450C3F
:100D9000B300440CB2003208A4003308A5000230AE
:100DA000B000B10152202C300320A9010530441CB1
:100DB0000301B2000030441C0301B3003208A40058
:100DC0003308A5000230B000B101522020300320CA
:100DD000DF300320433003208A110A122A2FFE300D
:100DE0000320C03003204D300320613003207830D1
:100DF00003202030032045300320783003202030AA
:100E0000032020300320A90103103D0CB3003C0C4B
:100E1000B2003208A4003308A5000230B000B101CE
:100E200052202C300320A90105303C1C0301B200E4
:100E300000303C1C0301B3003208A4003308A500B5
:100E40000230B000B101522020300320DF300320F7
:100E5000433003200730A300D030812064008A1182
:100E60000A1285198F2F8A110A12FA30C000C101A7
:100E70009230BC00FF30BD00FA30C200C301923096
:100E8000BE00FF30BF00FE3003200130032052308F
:100E90000320413003205A300320203003204D30FE
:100EA0000320693003206E30032069300320203096
:100EB00003206530032074300320203003204D30A0
:100EC0000320613003207830032069300320FE3096
:100ED0000320C030032020300320203003202030A6
:100EE000032020300320723003206530032061305E
:100EF00003206C30032069300320733003206530F9
:100F000003206530032020300320203003202030D0
:100F10000320203003200330A300E830812065291E
:100F200005108316051083120130A100F4308E20C5
:100F300083160514643083128D2064008A110A120E
:100F4000051CC82F8A110A12FE300320023003202C
:100F5000493003206E3003207430032065300320B5
:100F60007230032069300320653003207530032080
:100F700072300320203003206130032062300320D0
:100F800073300320653003206E300320743003205B
:100F90000130A10090308E208510831685108312B9
:100FA0000130A100F4308E20831685146430831242
:100FB0008D2064008A150A12851C0A288A110A12DB
:100FC000FE300320C030032045300320783003205A
:100FD0007430032065300320723003206930032011
:100FE0006530032075300320723003202030032049
:100FF000613003206230032073300320653003200A
:101000008A156E308A158A1103208A1574308A1168
:1010100003208A150130A10090308A118E208A1594
:1010200008000130CB00640009304B028A150A1217
:10103000031835288A150A1264008A150A124A18FC
:101040002B288A150A128A150A125B208A150A12A1
:101050008A150A1230288A150A1267208A150A1280
:101060000310CA0CCB0A031D132808000130CB0063
:10107000640009304B028A150A1203185A288A158F
:101080000A1264008A150A124A1850288A150A1290
:101090008A150A1274208A150A128A150A1255280E
:1010A0008A150A1280208A150A120310CA0CCB0A6C
:1010B000031D382808000510831605103C308A11DE
:1010C00083128D208A1583160514831208000510DB
:1010D0008316051083120000831605143C308A1114
:1010E00083128D208A1508008510831685103C30E8
:1010F0008A1183128D208A158316851483120800A5
:1011000085108316851083120000831685143C30E9
:101110008A1183128D208A1508000130CB006400EB
:1011200011304B028A150A120318A3288A150A12D5
:101130000310C90CC80C8A150A12BB208A150A12A2
:10114000CB0A031D8F2808000130CB00640011304A
:101150004B028A150A120318BA288A150A120310BC
:10116000C70CC60C8A150A12D1208A150A12CB0A9E
:10117000031DA6280800C917051083160510831241
:1011800000008316051464008A150A1283120518DC
:10119000CC288A150A12C9133C308A118D208A1571
:1011A0000800C71785108316851083120000831668
:1011B000851464008A150A1283128518E2288A159C
:1011C0000A12C7133C308A118D208A15080063006B
:0211D000E7280E
:02400E00753DFE
:00000001FF
